:100000000C941A060C945E060C945E060C945E0624
:100010000C945E060C945E060C945E060C945E06D0
:100020000C945E060C945E060C945D110C942F12D9
:100030000C9410200C945E060C945E060C945E06E4
:100040000C945E060C945E060C945E060C945E06A0
:100050000C945E060C9478200C945E060C945E065C
:100060000C945E060C945E060C945E060C945E0680
:100070000C945E060C945E060C945E060C945E0670
:100080000C945E060C945E060C945E060C945E0660
:100090000C945E060C945E060C945E060C945E0650
:1000A0000C945E060C945E060C945E069C12BE12C6
:1000B000AC13BE12AC1303132613AC137B138E13B5
:1000C000D116D116001700173F175F178F188F181A
:1000D0006A178F181A181A1880188F188F1889180D
:1000E0002718271827182718271827182718271818
:1000F0002718271827182718271827182718271808
:10010000371845184C1853185D1814001A000800C9
:100110001500170001001C0018000C00120013004D
:1001200004001600070009000A0001000B000D0082
:100130000E000F0033001D001B0006001900050013
:10014000E2001100100036003700380029002B00B3
:10015000E300E1002A00E0002C0001522D003400F1
:1001600028001E021F022F023002310201004B0044
:100170002400250026002502200221022602270253
:10018000350001004E002100220023002E02220231
:1001900023022F0030003502E20024021E001F005F
:1001A0002000310002544900E300E1002A00E00091
:1001B0002C000100370027002E0049004A005200A1
:1001C0004D004B000100520040004100420043003E
:1001D0004C00500051004F005100010051003D0003
:1001E0003E003F0044000100010001000100010049
:1001F000E20001003A003B003C0045000100010024
:10020000E300E1002A00E0002C000053010001009F
:1002100000500A44454255473A20656E61626C655C
:10022000642E0A005374617465206F6620726F77C4
:100230002025583A2025303136620A0048756D6114
:100240006E2D7265616461626C65206D61747269A6
:10025000782073746174653A0D0A004465626F75A5
:100260006E63696E672064656C61792072656D618B
:10027000696E696E673A2025580A005B735D004B12
:100280006579626F6172642073746172742E0A0002
:100290005B575D005B535D005B525D005B445D003E
:1002A0005B435D000E034100740072006500750041
:1002B00073000000180354006500630068006E00BE
:1002C0006F006D0061006E006300790000000403A0
:1002D000090409028D00050100A0FA0904000001CB
:1002E00003010100092111010001223F00070581DE
:1002F0000308000A09040100010301020009211199
:10030000010001224D000705820308000A090402CA
:10031000000103000000092111010001223600073D
:1003200005830308000A0904030002030000000912
:10033000211101000122200007058403200001078C
:100340000504032000010904040001030000000962
:100350002111010001223900070585031000011257
:1003600001100100000008EDFE60600100010200C4
:100370000105010906A101050719E029E715002576
:100380000195087501810205081901290595057572
:10039000019102950175039101050719002977154F
:1003A000002501957875018102C00631FF0974A10D
:1003B000010975150025FF9520750881020976153C
:1003C0000025FF952075089102C005010980A10153
:1003D000850216010026B7001A01002AB700751021
:1003E00095018100C0050C0901A1018503160100DA
:1003F000269C021A01002A9C02751095018100C0FA
:1004000005010902A1010901A10005091901290538
:10041000150025019505750181029501750381017E
:100420000501093009311581257F9502750881067E
:1004300009381581257F950175088106050C0A3854
:10044000021581257F950175088106C0C005010947
:1004500006A101050719E029E71500250195087592
:100460000181029501750881010508190129059589
:100470000575019102950175039101050719002980
:10048000FF150025FF950675088100C00A0025307C
:10049000325820006B6579626F6172645F726570BB
:1004A0006F72743A20004B6579626F617264204C00
:1004B0004544732073746174653A2025780A00649A
:1004C000656C5F6B65795F6269743A2063616E2762
:1004D000742064656C3A20253032580A00616464E7
:1004E0005F6B65795F6269743A2063616E2774207F
:1004F0006164643A20253032580A00290A002575C3
:10050000002F002575005D2800256400200025646B
:1005100000200025640020002564007C0025303286
:1005200058006D6F7573656B6579205B62746E7CC6
:10053000782079207620685D287265702F61636C61
:10054000293A205B006D6B5F776865656C5F746945
:100550006D655F746F5F6D6178203D2025640A00D2
:100560006D6B5F776865656C5F6D61785F737065F3
:100570006564203D2025640A006D6B5F74696D65BC
:100580005F746F5F6D6178203D2025640A006D6B9C
:100590005F6D61785F7370656564203D2025640A36
:1005A000006D6B5F696E74657276616C203D20250D
:1005B000640A006D6B5F64656C6179203D20256481
:1005C0000A006D6B5F776865656C5F74696D655F68
:1005D000746F5F6D6178203D2025640A006D6B5F4C
:1005E000776865656C5F6D61785F737065656420C1
:1005F0003D2025640A006D6B5F74696D655F746FE3
:100600005F6D6178203D2025640A006D6B5F6D6130
:10061000785F7370656564203D2025640A006D6B0A
:100620005F696E74657276616C203D2025640A00F6
:100630006D6B5F64656C6179203D2025640A000A5A
:1006400000257500363A20776865656C5F74696DC2
:10065000655F746F5F6D61783A20000A0025750050
:10066000353A20776865656C5F6D61785F7370659A
:1006700065643A20000A00257500343A2074696DDB
:10068000655F746F5F6D61783A20000A0025750020
:10069000333A206D61785F73706565643A20000AB3
:1006A00000257500323A20696E74657276616C2897
:1006B0006D73293A20000A00257500313A206465DF
:1006C0006C6179282A31306D73293A20000A092D8E
:1006D0002056616C756573202D0A004D3E004D2536
:1006E000643E20003F007365742064656661756C2C
:1006F000740A00433E200077686572652064656C6B
:1007000074613A20637572736F723D25642C207793
:100710006865656C3D25640A53656520687474706E
:100720003A2F2F656E2E77696B6970656469612E4B
:100730006F72672F77696B692F4D6F7573655F6B8C
:100740006579730A000A092D204D6F7573656B6515
:1007500079202D0A4553432F713A09717569740A3E
:10076000313A0964656C6179282A31306D73290A40
:10077000323A09696E74657276616C286D73290A64
:10078000333A096D61785F73706565640A343A09BC
:1007900074696D655F746F5F6D61780A353A0977CA
:1007A0006865656C5F6D61785F73706565640A3656
:1007B0003A09776865656C5F74696D655F746F5F32
:1007C0006D61780A0A703A097072696E74207661F8
:1007D0006C7565730A643A097365742064656661B3
:1007E000756C74730A75703A092B310A646F776EF1
:1007F0003A092D310A706775703A092B31300A7049
:1008000067646F776E3A092D31300A0A7370656537
:1008100064203D2064656C7461202A206D61785FDE
:100820007370656564202A20287265706561742084
:100830002F2074696D655F746F5F6D6178290A00A0
:100840003F004D3E2000433E20004C25640A0074CA
:10085000696D65725F636F756E743A202530346C14
:10086000580A006B6579626F6172645F6E6B726FBC
:100870003A2025580A006B6579626F6172645F697E
:10088000646C653A2025580A006B6579626F617265
:10089000645F70726F746F636F6C3A2025580A0042
:1008A000686F73745F6B6579626F6172645F6C65AA
:1008B000647328293A2025580A000A092D20537408
:1008C00061747573202D0A004743433A20342E3952
:1008D0002E32204156522D4C4942433A20312E3877
:1008E0002E31204156525F415243483A2061767280
:1008F000350A004F5054494F4E533A204C5546410B
:10090000204D4F5553454B45592045585452414B66
:10091000455920434F4E534F4C4520434F4D4D4179
:100920004E44204E4B524F20343039360A00425547
:10093000494C443A20313637313865662D64697246
:100940007479202832333A30383A3534204A756E7B
:100950002020392032303136290A005649443A20C5
:1009600030784645454428546563686E6F6D616E06
:10097000637929205049443A20307836303630287F
:1009800041747265757329205645523A203078308B
:100990003030310A00444553433A20712E6D2E6B9E
:1009A0002E206B6579626F617264206669726D7763
:1009B00061726520666F72204174726575730A00FA
:1009C0000A092D2056657273696F6E202D0A000A80
:1009D000092D20436F6E736F6C65202D0A455343BC
:1009E0002F713A09717569740A6D3A096D6F7573E3
:1009F000656B65790A000A092D204D6167696320DE
:100A00002D0A443A094465627567204D6573736128
:100A1000676520546F67676C650A583A094D6174C1
:100A2000726978204465627567204D6F6465205453
:100A30006F67676C65202D2053686F77206B657931
:100A40007072657373657320696E206D617472696D
:100A50007820677269640A4B3A094B6579626F6165
:100A6000726420446562756720546F67676C652007
:100A70002D2053686F77206B6579707265737320D2
:100A80007265706F72740A4D3A0944656275672029
:100A90004D6F75736520546F67676C650A563A0928
:100AA00056657273696F6E0A533A095374617475AF
:100AB000730A433A09416374697661746520436F30
:100AC0006E736F6C65204D6F64650A46312D46313B
:100AD000303A0953776974636820746F204C6179E8
:100AE000657220302D392028463130203D204C3091
:100AF000290A302D393A0953776974636820746F75
:100B0000204C6179657220302D390A4553433A09EA
:100B100053776974636820746F204C617965722023
:100B2000302028616C7465726E617465206B657924
:100B30002031290A47524156453A0953776974636F
:100B40006820746F204C6179657220302028616CB8
:100B50007465726E617465206B65792032290A5064
:100B6000415553453A094A756D7020746F20426FA4
:100B70006F746C6F616465722028526573657429A7
:100B80000A4E3A094E4B524F20546F67676C650A04
:100B9000003F004E4B524F3A206F66660A004E4BA4
:100BA000524F3A206F6E0A000A6D6F7573653A20D6
:100BB0006F66660A000A6D6F7573653A206F6E0A7C
:100BC000000A6B6579626F6172643A206F66660A2B
:100BD000000A6B6579626F6172643A206F6E0A0079
:100BE0000A6D61747269783A206F66660A000A6D50
:100BF00061747269783A206F6E0A000A64656275E2
:100C0000673A206F66660A000A64656275673A2073
:100C10006F6E0A000A0A4A756D70696E6720746FFC
:100C200020626F6F746C6F616465722E2E2E2000CF
:100C3000433E200011241FBECFEFDAE0DEBFCDBF60
:100C400004B603FE24C08091FE019091FF01A091A3
:100C50000002B09101028730904BA740B04BB9F42D
:100C60001092FE011092FF011092000210920102F8
:100C700014BE84B7877F84BF88E10FB6F894809351
:100C80006000109260000FBEE0E0F8E3099511E00B
:100C9000A0E0B1E0E8E9F2E502C005900D92A834C9
:100CA000B107D9F711E0A8E4B1E001C01D92AE3F51
:100CB000B107E1F70E94970E0C944A290C940000AA
:100CC000FF93EF93E0914801F0914901309709F0CB
:100CD0000995EF91FF910895FC018591803011F005
:100CE000EFDFFBCF0895FF27E0E230E247FF0CC0C3
:100CF000419597FF09C0EDE26095709580959095BC
:100D0000611D711D811D911D27FF02C0219530E3DA
:100D100050E2AA27660F771F881F991FAA1FA417E2
:100D200010F0A41B63955A95A9F7AA3008F0A95FA3
:100D3000A05DAF93F395611571058105910541F7AC
:100D4000ED3211F4EF93F395F21718F43F93F39506
:100D5000FBCF8F91B5DFFA95E1F70895E991F9910D
:100D60008591803021F0853219F0AADFF9CF0895FE
:100D700020E0E89455915532C1F3503311F4689452
:100D800055915A3348F4505390F3220F022E220FFC
:100D9000220F200D250FF4CF0EF421958991999102
:100DA000533619F3533729F1533559F1BC018827CC
:100DB0009927E8945C3621F489919991689455912A
:100DC000543639F446EF7EF077FF0DC08FEF9FEF7A
:100DD0000AC055374AE039F0583540E121F0523623
:100DE00042E009F00895FF93EF937DDFEF91FF91CB
:100DF000B7CFFF93EF93FC0181918030B9F360DFAF
:100E0000FBCFFF93EF9368DFF1CFDF93CF93CDB7A5
:100E1000DEB72596A3DFCF91DF9108950895089559
:100E20008EE097E0892B11F00C940E0708958FE067
:100E300097E0892B11F00C940F07089561110BC0F6
:100E4000FC018281882321F085EE0E94751503C084
:100E500085EE0E943D1680E090E0089581E00895BF
:100E600081E008950C94300708950F931F93CF935A
:100E7000DF938C01FC01C081D181CE010E94F31D62
:100E8000BE010E94E207EC01B8010E9432078823EC
:100E900009F48DC0F8018281882309F44AC0809149
:100EA000550181111FC0C431F0E5DF0709F051C0C1
:100EB0000E94340781E0809355010E944220909364
:100EC00054018093530110924C0110924E011092E4
:100ED0004D011092500110924F0110925201109248
:100EE000510165C080915301909154010E944E20A0
:100EF000883C910570F480914C01E82FF0E0EE0FF2
:100F0000FF1FE35BFE4FD183C0838F5F80934C0153
:100F10004EC0C43880E5D80721F0C538D04501F16E
:100F20003AC0F8018281882341F010924A0182E0A0
:100F30001EC0C438E0E5DE0759F580914A018111F1
:100F400006C086E20E94751586E20E943D1682E088
:100F50001CC0C438F0E5DF0741F3C538D045D9F4EB
:100F6000F8018281882331F010924B0180E20E94C7
:100F70008C161DC080914B01811106C087E20E9432
:100F8000751587E20E943D1680E20E9493160FC0FD
:100F9000C538D04529F381E080934A0180934B0105
:100FA000C801DF91CF911F910F910C942E0780E023
:100FB000DF91CF911F910F9108950C9410070C941D
:100FC000170708959BE0799FF00111249CE2899F07
:100FD000E00DF11D1124E60FF11DEE0FFF1FE65F7E
:100FE000FE4F859194910895880F991FFC01E65753
:100FF000F040859194910895880F991FFC01E65F58
:10100000FE4F8591949108950F931F93CF93DF9393
:10101000EC01811520E3920750F5C11580E2D80755
:1010200008F0C9C0CB3BD10590F4C83AD10508F00F
:1010300070C0C53AD10508F061C0C430D10508F0D0
:10104000DAC1219709F0D4C101E010E014C2CF3F0A
:10105000D10511F008F0CFC1C03FD10508F0A8C0FC
:10106000CE01805E9109089708F4C5C1C1C1C130A5
:1010700090E5D90709F4A8C050F5C0318FE4D8072E
:1010800070F4C11590E4D90708F09AC0C11521E3A6
:10109000D20708F0ADC1DD278E01106CECC1C1157F
:1010A000D04509F0A5C10E94FA188FEF94E32CE017
:1010B000815090402040E1F700C0000087E797E7AB
:1010C00090930108809300080E949D20D4C1C1150F
:1010D00097E5D90758F4C03121E5D20708F020C1BF
:1010E000C43180E5D80708F479C082C1CE01905799
:1010F0008115904108F07CC1DF7077C1C53AD105F8
:1011000009F47BC1C63AD10509F07AC102E810E4BE
:10111000B2C1C83AD10509F476C1C93AD10509F47A
:1011200075C1CA3AD10509F474C1CB3AD10509F4A5
:1011300073C1CC3AD10509F472C1CD3AD10509F495
:1011400071C1C03BD10509F470C1CE3AD10509F493
:101150006FC1CF3AD10509F46EC1C13BD10509F485
:101160006DC1C23BD10509F46CC1C33BD10509F483
:101170006BC1C43BD10509F46AC1C53BD10509F473
:1011800069C1C63BD10509F468C1C73BD10509F463
:1011900067C1C83BD10509F466C1C93BD10509F453
:1011A00065C1CA3BD10509F464C100E014E463C120
:1011B0008E01106560C1CE019F700E94FC075CC16A
:1011C000DF708E01106A57C182E192E00E946C06C6
:1011D0008091DF0181608093DF014DC10E94F42086
:1011E000811102C00E94DA200E94072190E09093B2
:1011F000FE018093FD01C23080E5D80721F4809183
:10120000FD01816086C0C43090E5D90721F480914A
:10121000FD0182607EC0C63020E5D20721F48091B6
:10122000FD01846076C0C83080E5D80719F480914C
:10123000FD0127C0CA3090E5D90721F48091FD0156
:10124000806167C0CC3020E5D20721F48091FD0198
:1012500080625FC0CE3080E5D80721F48091FD0127
:10126000806457C0C03190E5D90721F48091FD0119
:1012700080684FC0C23120E5D20729F48091FD017A
:101280008460886046C0C33080E5D80721F480912F
:10129000FD018E7F3EC0C53090E5D90721F48091D5
:1012A000FD018D7F36C0C73020E5D20721F4809143
:1012B000FD018B7F2EC0C93080E5D80719F48091DD
:1012C000FD0126C0CB3090E5D90721F48091FD01C6
:1012D0008F7E1FC0CD3020E5D20721F48091FD0123
:1012E0008F7D17C0CF3080E5D80721F48091FD01B4
:1012F0008F7B0FC0C13190E5D90721F48091FD01AA
:101300008F7707C0C331D04531F48091FD018B7FC9
:10131000877F8093FD018091FD010E940B21ABC06E
:101320008D2F99278F70992781309105D9F49E01CF
:101330002370332702C0880F991F2A95E2F79C6813
:101340008E0144E0000F111F4A95E1F7002713704A
:10135000802B912B53E0CC0FDD1F5A95E1F7C0761F
:10136000DD272FC08230910531F4DC2FCC278E0190
:10137000016F106A80C08330910569F4CE018370DB
:10138000992701E010E002C0000F111F8A95E2F7D3
:10139000C8019C680FC084309105B9F4CE018370F8
:1013A000992701E010E002C0000F111F8A95E2F7B3
:1013B000C8019A6823E0CC0FDD1F2A95E1F7C07EB3
:1013C000D7708C010C2B1D2B56C08530910531F444
:1013D000DC2FCC278E01046F106A4DC0069709F0F0
:1013E0004AC0CF71DD27DC2FCC278E01106243C0AD
:1013F00000E010E040C08E013EC001E810E43BC0B8
:1014000003E810E438C002EE14E435C009EE14E439
:1014100032C00AEE14E42FC005EB14E42CC006EB36
:1014200014E429C007EB14E426C00CEC14E423C038
:101430000DEC14E420C003E815E41DC00AE815E42F
:101440001AC002E915E417C004E915E414C001E26A
:1014500016E411C003E216E40EC004E216E40BC069
:1014600005E216E408C006E216E405C007E216E449
:1014700002C00AE216E4C801DF91CF911F910F91DB
:1014800008959BE0799FF00111249CE2899FE00D73
:10149000F11D1124E60FF11DEE0FFF1FE65FFE4F59
:1014A00085919491803E9105E0F4803C910558F53A
:1014B0008133910509F46FC048F48932910509F42C
:1014C00063C08A32910509F46DC072C089339105F9
:1014D000E9F082389105D1F08533910509F44DC0CA
:1014E00067C0833E910581F138F4803E9105B9F0E3
:1014F000823E9105D9F05CC0863E910561F1873E40
:101500009105A1F155C00E94F40708952091FD01B5
:1015100020FD02C021FF4CC080EE90E049C08091C8
:10152000FD0180FFF9CF89E390E042C08091FD0189
:1015300082FF0EC08091FD0184FF03C080E090E037
:1015400037C083EE90E034C08091FD0182FFF2CF7E
:1015500082EE90E02DC08091FD0183FF0BC0809151
:10156000FD0184FDEBCF87EE90E022C08091FD016C
:1015700083FFF5CF86EE90E01BC08091FD0185FFD3
:1015800007C089E290E014C08091FD0185FFF9CF8A
:1015900085E390E00DC08091FD0186FF07C08AE2DF
:1015A00090E006C08091FD0186FFF9CF81E390E0D5
:1015B0000E940408089508950C94DB0AE82FF0E0D7
:1015C000E05EFE4F8081E82FEF70F0E082958F7033
:1015D00021E030E0A90102C0440F551F8A95E2F7CF
:1015E00040A308950F931F93CF93DF9385B780682F
:1015F00085BF85B7806885BFC3E0D0E001E010E01B
:10160000FE01E05EFE4F8081E82FEF70F0E021A147
:1016100082958F70A80102C0440F551F8A95E2F78A
:10162000CA01822B81A38C2F0E94DE0A219740F7EA
:101630008AE090E061E070E0FC01EB5EFE4F20810B
:10164000E22FEF70F0E042A122952F70DB0102C083
:10165000AA0FBB1F2A95E2F79D01242B22A3019715
:1016600058F7DF91CF911F910F910C94DD07EF9206
:10167000FF920F931F93CF93DF930EE511E0C3E02A
:10168000EE24E394F12CD5E08C2F0E94DE0A8AE050
:1016900090E040E050E0FC01EB5EFE4F6081E62F01
:1016A000EF70F0E020A130E062956F7002C03595D8
:1016B00027956A95E2F720FD09C09701082E02C020
:1016C000220F331F0A94E2F7422B532B019718F78E
:1016D000F801929182918F018417950721F051832F
:1016E0004083D09300018C2F0E94DE0AC15060F627
:1016F0008091000187FD42C09091DF0190FF10C0F2
:10170000282F332727FD30953F938F938BE592E069
:101710009F938F930E9405070F900F900F900F904B
:101720008091000181508093000187FD07C08FE9FF
:101730009FE00197F1F700C0000020C080915C019C
:1017400090915D01909365018093640180915A01AD
:1017500090915B01909363018093620180915801A5
:10176000909159019093610180936001809156019D
:101770009091570190935F0180935E010E94DF0773
:1017800081E0DF91CF911F910F91FF90EF9008952D
:10179000E82FF0E0EE0FFF1FE25AFE4F80819181AB
:1017A0000895EF92FF920F931F93CF93DF93809151
:1017B000DF0180FF04C08CE392E00E946C060EE51E
:1017C00011E0C0E0D0E084E2E82E82E0F82E8091C3
:1017D000DF0180FF13C0F801808191810E94B71F53
:1017E0009F938F93DF93CF93FF92EF920E94050711
:1017F0000F900F900F900F900F900F9021960E5F0B
:101800001F4FC430D10519F7DF91CF911F910F9170
:10181000FF90EF9008950F931F93CF9306E611E08A
:10182000C0E0F801929182918F010E94951FC80F2C
:10183000F1E00E351F07A9F78C2FCF911F910F9163
:1018400008958091790108959FB7F89410926801E6
:101850009FBF9091F401943009F057C09091E90036
:101860009F703091EC00232F217030FD20E8922BE7
:1018700024E02093E9002091EB0020FF43C0209159
:10188000EE0027FF3FC020916601222321F0209126
:10189000E80025FF37C01092660126E03091E8008D
:1018A00035FD15C03091F401343061F53091EB0015
:1018B00035FD28C0215021F481E08093660122C0CB
:1018C000EFE9FFE03197F1F700C00000E7CF809328
:1018D000F1008091E80085FD0AC08091E80080FF5A
:1018E000FCCF8091E8008E778093E80006C08FB728
:1018F000F89421E0209368018FBF9F709093E900D6
:1019000080E008959F709093E9008FEF0895CF9342
:10191000DF9300D01F92CDB7DEB79C018091F40118
:10192000843019F593E099833B832A839093E900EF
:101930008FEF9091E800815095FD06C095ED9A9546
:10194000F1F700008111F5CF8091E80085FF0DC00F
:1019500040E050E063E070E0CE0101960E944D0F40
:101960008091E8008E778093E8000F900F900F90A1
:10197000DF91CF910895CF93DF9300D01F92CDB721
:10198000DEB72091F401243021F522E029839B83E6
:101990008A8383E08093E9008FEF9091E800815083
:1019A00095FD06C095ED9A95F1F700008111F5CFF0
:1019B0008091E80085FF0DC040E050E063E070E0FA
:1019C000CE0101960E944D0F8091E8008E778093A2
:1019D000E8000F900F900F90DF91CF910895209124
:1019E000F4012430F1F422E02093E9002FEF30914C
:1019F000E800215035FD06C035ED3A95F1F70000BD
:101A00002111F5CF2091E80025FF0BC040E050E008
:101A100065E070E00E944D0F8091E8008E77809322
:101A2000E8000895CF93DF932091F401243009F06A
:101A300048C0EC0180910B018823E1F080910C01FA
:101A40008823C1F085E08093E9008FEF9091E80052
:101A5000815095FD06C095E19A95F1F7000081113E
:101A6000F5CF8091E80085FF2CC040E050E060E1B8
:101A700070E017C081E08093E9008FEF9091E8005B
:101A8000815095FD06C095ED9A95F1F70000811102
:101A9000F5CF8091E80085FF14C040E050E068E099
:101AA00070E0CE010E944D0F8091E8008E77809308
:101AB000E80080E1FE01A9E6B1E001900D928A956F
:101AC000E1F7DF91CF91089580EA92E00E946C06E1
:101AD0008091F301811109C00E94E2100E943F1120
:101AE0008091E20084608093E20008958CE992E0A6
:101AF0000E946C061092F301089588E992E00C941C
:101B00006C0684E992E00C946C0680E992E00E94F5
:101B10006C060C940A20209167012F5F822F62E3EC
:101B20000E94DA28992319F02093670108951092F2
:101B3000670180916801882371F18091F4018430FC
:101B400041F58091E9008F702091EC00922F917007
:101B500020FD90E8892B94E09093E9009091EB00B0
:101B600090FF14C09091EE0097FF10C09091E80094
:101B700095FF03C01092F100F9CF9091E80090FF1B
:101B800005C09091E8009E779093E8008F70809355
:101B9000E90010926801089542E061EC81E00E9442
:101BA0005C1042E061EC82E00E945C1042E061EC7B
:101BB00083E00E945C1042E261EC84E00E945C10D1
:101BC00042E161EC85E00C945C108091F601833079
:101BD00009F455C030F4813071F0823009F48EC0C0
:101BE00008958A3009F47AC08B3009F460C08930D6
:101BF00009F09CC020C08091F501813A09F096C09F
:101C00008091E800877F8093E8008091F9019091AE
:101C1000FA01892B21F460E189E691E003C060E0DC
:101C200080E090E070E00E94980F8091E8008B7750
:101C30008093E80008958091F501813209F076C023
:101C40008091F9019091FA01009719F0049709F039
:101C50006DC08091E800877F8093E8008091E80064
:101C600082FD05C08091F4018111F8CF5FC08091A1
:101C7000F100809379018091E8008B7753C08091C7
:101C8000F501813A09F052C08091F9019091FA0171
:101C9000892B09F04BC08091E800877F8093E80092
:101CA0008091E80080FFFCCF80910B0136C08091CD
:101CB000F5018132D9F58091F9019091FA01892BD2
:101CC000A9F58091E800877F8093E8000E94911039
:101CD0008091F70180930B010C94FA188091F50123
:101CE000813221F58091E800877F8093E8000E948F
:101CF00091108091F80180937A0108958091F50107
:101D0000813AA1F48091E800877F8093E800809178
:101D1000E80080FFFCCF80917A018093F1008091F0
:101D2000E8008E778093E8000C949110089584B7B2
:101D3000877F84BF88E10FB6F8948093600010928B
:101D400060000FBE90E080E80FB6F89480936100C9
:101D5000909361000FBE0E9471140E94E2100E94D5
:101D60003F118091E20084608093E20084E29CE075
:101D70000E94901F78940E94C4130E94731481E003
:101D800091E00E94DF138FE792E00E946C06809141
:101D9000F401853089F48BE792E00E946C060E9482
:101DA000D11F8091F201882391F30E94FC1F8823A8
:101DB00071F30E94370FEBCF0E949714E8CF292FC1
:101DC000332723303105C9F064F42130310581F027
:101DD0002230310509F043C08DE890E022ED32E079
:101DE00042C021323105F1F02232310541F137C0D4
:101DF00082E190E02FE533E036C0992781309105EC
:101E000041F08230910541F0892B49F5EEECF2E08A
:101E100005C0E4EBF2E002C0E4EAF2E0849190E075
:101E20009F0121C06530D8F4E62FF0E0EE0FFF1FD0
:101E3000ED5CFE4F2081318189E090E014C0653077
:101E400070F470E0FB01EE0FFF1FE75DFE4F208195
:101E50003181FB01EC5DFE4F808190E004C080E0A9
:101E600090E020E030E0FA0131832083089580E1A2
:101E700089BD82E189BD09B400FEFDCF8091D80003
:101E80008F7D8093D8008091E00082608093E00095
:101E90008091E00081FDFCCF0895CF92DF92EF9218
:101EA000FF920F931F93CF93DF93EC018B016A0195
:101EB0000E94B010811133C0C114D10439F0F60171
:101EC00080819181081B190BC80FD91FE12CF12CBF
:101ED0000115110519F18091E80085FD16C080916A
:101EE000E8008E778093E800C114D10449F0F60130
:101EF00080819181E80EF91EF182E08285E00FC0B9
:101F00000E94B010882321F30AC089918093F100C8
:101F100001501109FFEFEF1AFF0ADACF80E0DF91DD
:101F2000CF911F910F91FF90EF90DF90CF90089588
:101F30002091FB013091FC012617370748F061150D
:101F4000710539F42091E8002E772093E80001C054
:101F5000B90140E061157105A9F12091F401222336
:101F600009F443C0253009F442C02091E80023FD64
:101F700040C02091E80022FD32C02091E80020FFFF
:101F8000E9CF4091F3002091F20030E0342BFC01C6
:101F9000CF016115710559F02830310540F4819168
:101FA0008093F100615071092F5F3F4FF1CF41E005
:101FB0002830310509F040E02091E8002E77209389
:101FC000E800C8CF4111C9CF0AC08091F40188232D
:101FD00061F0853061F08091E80083FD0AC0809156
:101FE000E80082FFF2CF80E0089582E0089583E068
:101FF000089581E008952091FB013091FC0126179E
:10200000370748F06115710539F42091E8002E7703
:102010002093E80001C0B901FC0120E061157105C1
:1020200091F18091F401882309F440C0853009F4CE
:102030003FC08091E80083FD3DC08091E80082FDB3
:102040002FC08091E80080FFE9CF2091F3008091BC
:10205000F20090E0922B6115710559F088309105DE
:1020600040F424912093F10031966150710901965A
:10207000F2CF21E0089709F020E08091E8008E7708
:102080008093E800CBCF2111CCCF0AC08091F4011E
:10209000882361F0853061F08091E80083FD0AC0FB
:1020A0008091E80082FFF2CF80E0089582E00895F9
:1020B00083E0089581E00895982F973058F5909324
:1020C000E900981739F07091EC002091ED005091E3
:1020D000F00003C0242F762F50E021FF19C030916B
:1020E000EB003E7F3093EB003091ED003D7F30936D
:1020F000ED003091EB0031603093EB007093EC0019
:102100002093ED005093F0002091EE0027FF07C0D0
:102110009F5FD3CF8F708093E90081E0089580E0C6
:1021200008958091F50187FF11C08091E80082FD3C
:1021300005C08091F4018111F8CF11C08091E800B1
:102140008B770BC08091F401882349F08091E800DF
:1021500080FFF8CF8091E8008E778093E8000895A3
:102160002091E4003091E50095E64091EC00842F49
:10217000817040FF22C08091E80080FD1CC08091EA
:10218000F401882391F0853091F08091EB0085FD7A
:1021900010C04091E4005091E5004217530729F325
:1021A0009A01915011F784E0089582E0089583E048
:1021B000089581E0089580E008954091E80042FF8D
:1021C000DECF08950E9450110E945811E0EEF0E019
:1021D000808181608083E8EDF0E080818F7780836B
:1021E00019BCA7EDB0E08C918E7F8C9380818F7E9F
:1021F00080831092F30108950F931F93CF93DF9381
:102200000E9450110E945811C8EDD0E088818F774C
:10221000888388818068888388818F7D888319BCC2
:102220001092F4011092F0011092F2011092F1015B
:1022300000EE10E0F80180818B7F808388818160CF
:10224000888342E060E080E00E945C10E1EEF0E014
:1022500080818E7F8083E2EEF0E0808181608083E8
:10226000808188608083F80180818E7F808388816F
:1022700080618883DF91CF911F910F910895E8EDE0
:10228000F0E080818F7E8083E7EDF0E080818160E7
:10229000808384E082BF81E08093F3010C94FC1082
:1022A000E8EDF0E080818E7F80831092E200089557
:1022B0001092DA001092E10008951F920F920FB66B
:1022C0000F9211242F933F934F935F936F937F93BC
:1022D0008F939F93AF93BF93EF93FF938091E10010
:1022E00082FF0BC08091E20082FF07C08091E10075
:1022F0008B7F8093E1000E948B0D8091DA0080FF3C
:102300001FC08091D80080FF1BC08091DA008E7FB3
:102310008093DA008091D90080FF0DC080E189BDF3
:1023200082E189BD09B400FEFDCF81E08093F40114
:102330000E94640D05C019BC1092F4010E94760D34
:102340008091E10080FF19C08091E20080FF15C0FC
:102350008091E2008E7F8093E2008091E2008061B4
:102360008093E2008091D80080628093D80019BCED
:1023700085E08093F4010E94810D8091E10084FF4B
:1023800030C08091E20084FF2CC080E189BD82E1F1
:1023900089BD09B400FEFDCF8091D8008F7D809368
:1023A000D8008091E1008F7E8093E1008091E2006F
:1023B0008F7E8093E2008091E20081608093E20052
:1023C0008091F001882311F084E007C08091E30040
:1023D00087FD02C081E001C083E08093F4010E9488
:1023E000850D8091E10083FF29C08091E20083FF89
:1023F00025C08091E100877F8093E10082E0809397
:10240000F4011092F0018091E1008E7F8093E10051
:102410008091E2008E7F8093E2008091E2008061F3
:102420008093E20042E060E080E00E945C108091D6
:10243000F00088608093F0000E947D0DFF91EF9185
:10244000BF91AF919F918F917F916F915F914F91CC
:102450003F912F910F900FBE0F901F9018951F92D4
:102460000F920FB60F9211242F933F934F935F93C8
:102470006F937F938F939F93AF93BF93CF93DF938C
:10248000EF93FF93C091E900CF708091EC00D82FBB
:10249000D17080FDD0E81092E9008091F000877F34
:1024A0008093F00078940E9473121092E90080915A
:1024B000F00088608093F000CD2BCF70C093E900CE
:1024C000FF91EF91DF91CF91BF91AF919F918F914C
:1024D0007F916F915F914F913F912F910F900FBE20
:1024E0000F901F9018951F93CF93DF93CDB7DEB752
:1024F000AA970FB6F894DEBF0FBECDBFE5EFF1E0AF
:1025000088E08E0F9091F10091938E13FBCF0E9483
:10251000E50D8091E80083FF1FC18091F501909146
:10252000F601492F50E04A30510508F015C1FA0173
:10253000EA5AFF4F0C94FA28803881F0823809F06B
:102540000BC18091F9018F708093E9008091EB00BD
:1025500085FB882780F91092E90006C08091F1017F
:102560009091F201911182609091E800977F909391
:10257000E8008093F1001092F100C8C0282F2D7F51
:1025800009F0EAC0882319F0823061F0E5C080913B
:10259000F701813009F0E0C0933009F080E08093CA
:1025A000F2012BC08091F701811127C08091F901C0
:1025B0008F7009F4D1C08093E9002091EB0020FFD7
:1025C0001CC0933021F48091EB00806214C0909184
:1025D000EB0090619093EB0021E030E0A90102C094
:1025E000440F551F8A95E2F74093EA001092EA00E3
:1025F0008091EB0088608093EB001092E90080915D
:10260000E800877F86C08111A7C01091F7011F776E
:102610008091E3008078812B8093E3008091E80033
:10262000877F8093E8000E9491108091E80080FFEE
:10263000FCCF8091E30080688093E300111102C019
:1026400082E001C083E08093F40186C0805882302C
:1026500008F082C08091F7019091F8018C3D53E021
:10266000950779F583E08A838AE289834FB7F894E6
:10267000DE01139620E03EE051E2E32FF0E05093BC
:102680005700E49120FF03C0E295EF703F5FEF70C9
:102690008E2F90E0EA3010F0C79601C0C0968D935F
:1026A0009D932F5F243149F74FBF8091E800877FCA
:1026B0008093E8006AE270E0CE0101960E94980FD4
:1026C00014C0AE014F5F5F4F6091F9010E94DF0EB1
:1026D000BC01009709F440C09091E800977F909367
:1026E000E80089819A810E94FB0F8091E8008B7736
:1026F0008093E80031C0803879F58091E800877FC9
:102700008093E8008091F0018093F1008091E800CF
:102710008E778093E8000E9491101EC081111CC02A
:102720009091F7019230C0F48091E800877F809308
:10273000E8009093F0010E9491108091F0018111C6
:1027400006C08091E30087FD02C081E001C084E003
:102750008093F4010E94CC0D8091E80083FF0AC0B1
:102760008091E800877F8093E8008091EB00806291
:102770008093EB00AA960FB6F894DEBF0FBECDBFD4
:10278000DF91CF911F910895CF938091F401882319
:10279000A1F0C091E900CF709091EC00892F817079
:1027A00090FD80E8C82B1092E9008091E80083FD3D
:1027B0000E947312CF70C093E900CF910895909357
:1027C000800180937F010895E0917F01F091800165
:1027D000309721F00190F081E02D099480E0089578
:1027E000EF92FF920F931F93CF93DF93E0917F01BE
:1027F000F09180013097B1F18C010280F381E02DDE
:1028000009958091DF0182FF2DC080FF04C084E91B
:1028100094E00E946C06E80110E18EE8E82E84E066
:10282000F82E8091DF0180FF0BC088811F928F936B
:10283000FF92EF920E9405070F900F900F900F905C
:10284000115021961111EDCF8091DF0180FF0AC058
:102850008CE894E0DF91CF911F910F91FF90EF9062
:102860000C946C06DF91CF911F910F91FF90EF9028
:102870000895E0917F01F0918001309721F004806C
:10288000F581E02D0994089520917D0130917E011C
:102890008217930771F090937E0180937D01E09100
:1028A0007F01F0918001309721F00680F781E02DC3
:1028B0000994089520917B0130917C018217930740
:1028C00071F090937C0180937B01E0917F01F09106
:1028D0008001309721F00084F185E02D099408955E
:1028E00008950C9470140E9439200E94F20A0C94EE
:1028F000BF20CF93DF931F92CDB7DEB79091DF015A
:1029000092FF10C090FF0EC01F928F9326EA34E012
:102910003F932F9389830E9405070F900F900F908C
:102920000F9089810F90DF91CF910C94DC0A5F9218
:102930006F927F928F929F92AF92BF92CF92DF92CF
:10294000EF92FF920F931F93CF93DF9300D000D0AD
:102950001F92CDB7DEB70E94370B9AE8C92E91E0DF
:10296000D92E03E010E0AA24A394B12C502E802F7E
:102970000E94C80B4C01F601729062906F016826AC
:10298000792661147104A1F40150110978F78FEFD1
:1029900089838A831B820E9442208160782F9D83D5
:1029A0008C8349815A816B818D810E94471538C083
:1029B0008091DF0181FD0E94D10B2AE030E075019A
:1029C000022E02C0EE0CFF1C0A94E2F7C70186211A
:1029D0009721892B09F129835A828E209F2091E02B
:1029E000892809F490E09B830E9442208160782F1F
:1029F0009D838C8349815A816B818D810E9447150B
:102A0000000F111FF801EE57FE4F80819181E826DB
:102A1000F926F182E08204C02150310980F6B4CF5A
:102A20000E940C23109181010E94E4131817D1F029
:102A30000E94E413809381010F900F900F900F90EC
:102A40000F90DF91CF911F910F91FF90EF90DF904A
:102A5000CF90BF90AF909F908F907F906F905F903E
:102A60000C9479140F900F900F900F900F90DF91AE
:102A7000CF911F910F91FF90EF90DF90CF90BF907B
:102A8000AF909F908F907F906F905F900895CF93BD
:102A9000DF93CDB7DEB72B970FB6F894DEBF0FBE2E
:102AA000CDBF4F83588769877A878B87DE01119660
:102AB00086E0FD0111928A95E9F785E0FE013796DF
:102AC00001900D928A95E1F749815A816B817C8151
:102AD0008D819E810E94981B2B960FB6F894DEBFC5
:102AE0000FBECDBFDF91CF910895CF93882309F416
:102AF000C2C0C82F823859F40E94E41381FDBBC0C4
:102B000089E30E94721E0E94611F89E30CC0833812
:102B100079F40E94E41380FDAEC083E50E94721E2A
:102B20000E94611F83E50E94C51ECF910C94611F16
:102B3000843859F40E94E41382FD9DC087E40E940A
:102B4000721E0E94611F87E4EECF8CEF8C0F813ADA
:102B500048F48C2F0E94632681118DC08C2F0E9417
:102B6000721EE3CF80E28C0F883048F4C77081E09A
:102B700001C0880FCA95EAF70E941A1FD6CF8BE5CD
:102B80008C0F833078F4C53A29F0C63A31F083E8E7
:102B900090E005C081E890E002C082E890E0CF912B
:102BA0000C94441488E58C0F833108F064C0C83A53
:102BB00039F1C93A41F1CA3A49F1CB3A51F1CC3A2B
:102BC00059F1CD3A61F1C03B69F1CE3A71F1CF3A9A
:102BD00079F1C13B81F1C23B89F1C33B91F1C43B27
:102BE00099F1C53BA1F1C63BA9F1C73BB1F1C83B87
:102BF000B9F1C93BC1F1CA3BC9F180E090E038C0EE
:102C000082EE90E035C089EE90E032C08AEE90E02E
:102C10002FC085EB90E02CC086EB90E029C087EBBD
:102C200090E026C08CEC90E023C08DEC90E020C0BA
:102C300083E891E01DC08AE891E01AC082E991E042
:102C400017C084E991E014C081E292E011C083E2F0
:102C500092E00EC084E292E00BC085E292E008C0F0
:102C600086E292E005C087E292E002C08AE292E04A
:102C7000CF910C945A14CF910895882309F44BC036
:102C8000823859F40E94E41381FF45C089E30E9411
:102C9000721E0E94611F89E30CC0833871F40E9488
:102CA000E41380FF38C083E50E94721E0E94611FFA
:102CB00083E50E94C51E0C94611F843859F40E945C
:102CC000E41382FF28C087E40E94721E0E94611FE5
:102CD00087E4EFCF9CEF980F913A58F390E2980F6A
:102CE000983050F4877091E001C0990F8A95EAF707
:102CF000892F0E94201FDFCF9BE5980F933020F48F
:102D000080E090E00C944414885A833120F480E0F1
:102D100090E00C945A140895882321F00E941A1F01
:102D20000C94611F0895882321F00E94201F0C94A9
:102D3000611F08957F928F929F92AF92BF92CF9220
:102D4000DF92EF92FF920F931F93CF93DF931F9227
:102D5000CDB7DEB77C01C62E772EFC01058102952A
:102D60000F70128111110E94371F0E946B1E882361
:102D700079F0112369F080E28C0D883048F082E010
:102D80000E94541E0E946B1E91E0D82ED92601C0CD
:102D9000D12CE72DE295EF70F0E0E05AFF4F0C9454
:102DA000FA28872D807F072D0F70882311F0029558
:102DB000007F112389F0002309F498C180E28C0D73
:102DC000883020F4802F0E941A1F03C0802F0E9499
:102DD0002A1F0E94611F8AC18C2D0E943D1600236C
:102DE00009F49DC180E28C0D883020F4802F0E9470
:102DF000201F03C0802F0E94301F0E94611F8FC1BF
:102E0000872D807F972D9F70803211F4892F03C00A
:102E1000892F8295807FCC2021F0F1E0CF16A1F0A0
:102E20001DC0112339F0002319F1013009F50E946A
:102E30004A1F75C1002319F0013009F470C189835C
:102E40000E944D1F898110C1112321F0063008F026
:102E500066C10EC0053008F062C106C1112359F0E9
:102E6000002331F0F701958190FF40C19F70958359
:102E70000E948C1654C1002309F4F6C03DC1872D71
:102E800086958695837090E0009719F0019761F020
:102E900046C1112321F08C2D972D937002C080E044
:102EA00090E00E9444143BC1112321F08C2D972DFA
:102EB000937002C080E090E00E945A1430C18C2DC3
:102EC000112319F00E94922102C00E94FA210E944F
:102ED0007F2225C1872D837009F052C011111FC1B7
:102EE0008C2D829586958770880F880F9C2D9F70FA
:102EF000892E912CA12CB12C082E04C0880C991C71
:102F0000AA1CBB1C0A94D2F7C4FE14C00FE010E048
:102F100020E030E0B901A80104C0440F551F661F2E
:102F2000771F8A95D2F7CB01BA016095709580958D
:102F3000909503C060E070E0CB01272D2695269583
:102F4000237030E02230310569F02330310589F0FB
:102F5000682979298A299B292130310571F00E943D
:102F6000E01CDDC0682979298A299B290E94FC1C64
:102F7000D6C00E94E01CC501B4010E94C41CCFC091
:102F8000112319F0872D817001C08695882309F4DB
:102F9000C6C08C2D829586958770880F880F9C2DD2
:102FA0009F70892E912CA12CB12C082E04C0880C66
:102FB000991CAA1CBB1C0A94D2F7C4FE14C00FE0D3
:102FC00010E020E030E0B901A80104C0440F551F13
:102FD000661F771F8A95D2F7CB01BA01609570956D
:102FE0008095909503C060E070E0CB01272D269579
:102FF00026952370422F50E04230510569F043304E
:10300000510589F0682979298A299B294130510580
:1030100071F00E94BA1D83C0682979298A299B29E9
:103020000E94D61D7CC00E94BA1DC501B4010E9439
:103030009E1D75C08C2D90E0FC01E05EF109E5312C
:10304000F10508F04FC0E059FF4F0C94FA280C2D01
:103050000F70872D8F71112321F00E94371D802F53
:1030600007CF0E94581D802F0E94931658C011232D
:1030700041F0053008F053C0872D8F710E947D1DEF
:103080004EC0063008F04BC0F7CF112339F0872D22
:103090008F710E94371D43C01123C9F3872D8F7193
:1030A0000E94581D3CC0112329F0872D8F710E946A
:1030B000221D35C00E94181D32C0112351F0172D5A
:1030C0001F71812F0E94371D63E0812F0E944B1ECC
:1030D00026C081E00E94541E023008F182E00E9466
:1030E000541E1DC0112331F0002389F28C2D0E9443
:1030F000751515C0002391F28C2D0E943D160FC04E
:10310000472D4F706C2DC7010E941E070E943C1C6A
:1031100006C0472D4F706C2DC7010E94E107DD20CE
:10312000F9F00E94471E80FD1BC0F70112820E9429
:10313000411E0E94371DC7010E94BF180E94411EF8
:103140000F90DF91CF911F910F91FF90EF90DF9043
:10315000CF90BF90AF909F908F907F900C94581D10
:103160000F90DF91CF911F910F91FF90EF90DF9023
:10317000CF90BF90AF909F908F907F9008950F93C6
:103180001F93CF93DF93EC01888199812B813C8140
:10319000232BB9F09F3F11F48F3F99F0CE010E948D
:1031A0003507882371F0688179818A810E943D1EEC
:1031B0008C010E94F21D0E94B91CB801CE010E9430
:1031C0009A16DF91CF911F910F9108950E94371F9A
:1031D0000E94471F0E940C1F0E94611F0E94B22381
:1031E0000E947F2280E090E00E94441480E090E002
:1031F0000C945A140E94271F0C94E6180E94321E49
:10320000292F22952F7030E02C3031054CF42A30D4
:1032100031056CF42250310922303105A8F407C081
:103220002C30310569F02F30310551F00DC0803F51
:1032300069F018F4803E40F409C0843F29F406C0C8
:1032400093FB882780F9089580E0089581E0089530
:10325000CF93DF9300D000D01F92CDB7DEB70F9091
:103260000F900F900F900F90DF91CF910895CF9313
:10327000DF9300D000D000D0CDB7DEB726960FB6D2
:10328000F894DEBF0FBECDBFDF91CF9108951F939D
:10329000CF93DF93C0918A0116E080918B01C8170C
:1032A00099F0D0E01C9FF0011D9FF00D1124E45710
:1032B000FE4F4081518162817381848195810E949A
:1032C00037192196C770E9CFDF91CF911F910895EB
:1032D0004091BC015091BD016091BE017091BF0150
:1032E0008091C0019091C1010C9437198091C10166
:1032F00082958F7009F054C08091BE01882309F433
:103300004FC080918A01A0918B016091BC017091A6
:10331000BD014091BF015091C001B6E08A1709F488
:103320003FC090E041155105C1F17F3F11F46F3F5F
:10333000A1F1B89FF001B99FF00D1124E457FE4FA1
:10334000218172132AC02081621327C0228121119A
:1033500024C0238134812417350710F4215031090A
:10336000241B350B283C3105C0F42091C1012F707E
:1033700020612093C10126E0289FF001299FF00DD4
:103380001124EF56FE4F80818F70806180838CEB1B
:1033900091E00E94BF180C94471901968770BECF28
:1033A0000895CF92DF92EF92FF920F931F93CF93E6
:1033B000DF93CDB7DEB762970FB6F894DEBF0FBECE
:1033C000CDBF8C0185E0F801DE011D9601900D92C4
:1033D0008A95E1F7D8014C9111965C91119712965C
:1033E0006C9112971396CD90DC9014973091BC019C
:1033F0007091BD018091BF019091C001009709F4C7
:103400006BC17F3F19F43F3F09F466C1E090BE01F4
:10341000EE2009F4C0C02091C101C816D90628F0D9
:10342000F601E81BF90BCF0104C0809590958C0D37
:103430009D1DFF24F394883C910578F0F12C207FAA
:1034400009F0C6C07C2DD98AC88A89890E942819AA
:103450008CEB91E00E94BF18B1C0822F807F09F0F1
:1034600046C0751314C0341312C0611110C02F7000
:1034700020612093C1010E9468198CEB91E00E94A9
:10348000BF188091C101D80115968C932EC0CD280C
:1034900019F15F3F11F44F3FF9F0F62E61111CC096
:1034A00080918A0120918B0136E0821709F45AC07D
:1034B00090E0389FF001399FF00D1124E457FE4F42
:1034C0007181571306C07081471303C07281711157
:1034D00003C001968770E9CFF62E662309F418C160
:1034E0008091C10181608093C101F12C11C17513DC
:1034F00008C0341306C0611104C08091C101D80115
:10350000C3C04D875E878D859E856A8B0E94FE189D
:103510006A898823E1F16623D1F12091C101822FCC
:1035200082958F7090E0029774F08091BC01909129
:10353000BD0198878F831986DB86CA862C87CE01CA
:1035400007960E94BF1886E0F801ACEBB1E001904D
:103550000D928A95E1F70E9476190E946819FF245E
:10356000F394D6C04D875E878D859E850E94321E5E
:10357000292F22952F7030E0223031050CF0BCC08D
:103580009F7009F0B6C0805E883008F4C1C0C801E1
:103590000E94BF18E4CFC816D90608F453C0F6013C
:1035A000E81BF90BCF01883C910508F450C0F12CC1
:1035B0007C2DD98AC88A89890E942819ECEBF1E010
:1035C00086E0DF011D928A95E9F70E946819A0C084
:1035D000751314C0341312C0611110C08091C10161
:1035E000F8018583C8010E94BF1886E0ECEBF1E08A
:1035F000DF011D928A95E9F7FE2C8AC04D875E8710
:103600008D859E856A8B0E94FE186A89882309F43D
:10361000BECF662309F4BBCF2091C101822F8295D2
:103620008F7090E002970CF48ECF8091BC01909146
:10363000BD019A8389831B82DD82CC822E83CE01D9
:1036400001967FCF809590958C0D9D1DACCFF62E69
:10365000662309F49CCF75132EC034132CC020911F
:10366000C10120FD1FC0822F82958F70D9F0D80133
:1036700015962C9315978F3049F08F5F982F929560
:10368000907F822F8F70892B15968C93C8010E9492
:10369000BF1886E0F801ACEBB1E001900D928A957D
:1036A000E1F793CF86E0F801ACEBB1E001900D9229
:1036B0008A95E1F72DC04D875E878D859E850E9496
:1036C000FE18811140CF8091C10181608093C101BA
:1036D000C8010E94BF181CC0662309F458CF4D874B
:1036E0005E878D859E850E94FE18882309F44FCF42
:1036F0002ACF811148CF0CC0243031050CF047CFC0
:103700009F7009F440CFF8019581907F09F03BCF7D
:103710008F2D62960FB6F894DEBF0FBECDBFDF913E
:10372000CF911F910F91FF90EF90DF90CF90089570
:103730001F93CF93DF93CDB7DEB72C970FB6F894D6
:10374000DEBF0FBECDBF4F83588769877A878B87CF
:103750009C87CE0107960E94D119882369F08F813A
:1037600098852A853B85232BF1F19F3F09F063C0A3
:103770008F3F09F060C037C086E0FE013796DE015A
:10378000119601900D928A95E1F76F817885EA850F
:10379000FB85309741F17F3F11F46F3F21F120917C
:1037A0008B0130E0C90101968770992740918A0109
:1037B00050E08417950709F447C069837A83FD8335
:1037C000EC8396E0929FD001939FB00D1124A457F3
:1037D000BE4FFE01319601900D929A95E1F78093CC
:1037E0008B010E94471916E080918A0190918B010C
:1037F0008917C1F1189FC001112484579E4F0E9460
:10380000D119882379F1E0918A011E9FF0011124DA
:10381000E457FE4F4081518162817381848195819B
:103820000E94371980918A0190E00196877099274C
:1038300080938A01D9CF4F81588569857A858B8598
:103840009C850E943719CFCF0E94FA1810928B01E5
:1038500010928A01ECEBF1E086E0DF011D928A957F
:10386000E9F7C1CF2C960FB6F894DEBF0FBECDBFDF
:10387000DF91CF911F910895EF92FF920F931F93C5
:10388000CF93DF938C01009709F46CC0F12CEE24E8
:10389000E394E8012196F8018491843740F4843060
:1038A00008F051C0813081F0823019F15BC085375A
:1038B00009F444C0A8F19CE7980F903708F052C073
:1038C0008F770E943D1641C00E5F1F4FFE01C491CD
:1038D00080E28C0F883048F4C7708E2D01C0880FAD
:1038E000CA95EAF70E943A1F14C08C2F0E947515E2
:1038F0002DC00E5F1F4FFE01C49180E28C0F8830F7
:1039000058F4C7708E2D01C0880FCA95EAF70E943F
:10391000401F0E94611F1AC08C2F0E943D1616C0C6
:103920000E5F1F4FFE01C491CC2381F08FE99FE011
:103930000197F1F700C00000C150F6CF0E5F1F4F96
:10394000FE01F49003C00E9475158E018F2D88230F
:1039500009F49FCFEFE9FFE03197F1F700C00000D5
:103960008150F5CFDF91CF911F910F91FF90EF9094
:10397000089508956093C6017093C7018093C801AC
:103980009093C9010C94E6180F931F930091C60100
:103990001091C7012091C8013091C901DC01CB0110
:1039A000802B912BA22BB32B8093C6019093C70140
:1039B000A093C801B093C9011F910F910C94E61810
:1039C0000F931F930091C6011091C7012091C80168
:1039D0003091C901DC01CB0180239123A223B323C1
:1039E0008093C6019093C701A093C801B093C90109
:1039F0001F910F910C94E6180F931F930091C6012D
:103A00001091C7012091C8013091C901DC01CB019F
:103A100080279127A227B3278093C6019093C701DF
:103A2000A093C801B093C9011F910F910C94E6189F
:103A30001092C2011092C3011092C4011092C501EC
:103A40000C94E61841E050E060E070E004C0440FE0
:103A5000551F661F771F8A95D2F74093C201509376
:103A6000C3016093C4017093C5010C94E61841E052
:103A700050E060E070E004C0440F551F661F771FE0
:103A80008A95D2F78091C2019091C301A091C4019F
:103A9000B091C501482B592B6A2B7B2B4093C20157
:103AA0005093C3016093C4017093C5010C94E61850
:103AB00041E050E060E070E004C0440F551F661F15
:103AC000771F8A95D2F740955095609570958091B3
:103AD000C2019091C301A091C401B091C5014823D6
:103AE00059236A237B234093C2015093C3016093FF
:103AF000C4017093C5010C94E61841E050E060E009
:103B000070E004C0440F551F661F771F8A95D2F7D7
:103B10008091C2019091C301A091C401B091C501EF
:103B2000482759276A277B274093C2015093C30136
:103B30006093C4017093C5010C94E6180F931F9312
:103B40000091C2011091C3012091C4013091C501BF
:103B5000DC01CB01802B912BA22BB32B8093C201D4
:103B60009093C301A093C401B093C5011F910F911D
:103B70000C94E6180F931F930091C2011091C3019A
:103B80002091C4013091C501DC01CB018023912338
:103B9000A223B3238093C2019093C301A093C401D5
:103BA000B093C5011F910F910C94E6180F931F93CA
:103BB0000091C2011091C3012091C4013091C5014F
:103BC000DC01CB0180279127A227B3278093C20174
:103BD0009093C301A093C401B093C5011F910F91AD
:103BE0000C94E6180895CF92DF92EF92FF920F9314
:103BF0001F93CF93DF938C01C090C601D090C70173
:103C0000E090C801F090C9018091C2019091C30178
:103C1000A091C401B091C501C82AD92AEA2AFB2A79
:103C2000CFE1D0E0D701C6010C2E04C0B695A79510
:103C3000979587950A94D2F780FF06C0B8018C2F1C
:103C40000E94410A019721F4219760F780E001C0AA
:103C50008C2FDF91CF911F910F91FF90EF90DF900C
:103C6000CF900895CF93DF93EC010E94F31DBE0126
:103C70000E94410ADF91CF910895CB010E94321E2C
:103C800008958091CA0185958595859508958091BF
:103C9000CA018770089598E0899F90011124262B0E
:103CA0002093CA010C94371D2091CA01809582236C
:103CB0008093CA01982F977069F430E0482F5527F8
:103CC00047FD50952417350729F0859585958595ED
:103CD0000C94581D08959091CA01977081E009F4E1
:103CE00080E0089590910B01992321F090910C01AF
:103CF000911109C020910D0130910E01F901329608
:103D00009FEF40E030C0982F9695969596959F30FE
:103D1000A0F4E0910D01F0910E01E90FF11D877003
:103D200021E030E0A90102C0440F551F8A95E2F757
:103D3000CA019181892B818308959091DF0190FFC1
:103D400023C01F928F938DED94E09F938F930E94D9
:103D500005070F900F900F900F9008959F3F39F037
:103D60004F5F4E3041F051915813F8CF0DC05111B3
:103D7000F7CF942FF5CF9F3F39F0F901E90FF11DEF
:103D800097FDFA9582830895089590910B019923E8
:103D900021F090910C01911109C020910D013091F9
:103DA0000E01F9013296205F3F4F30C0982F969553
:103DB000969596959F30A8F4E0910D01F0910E0133
:103DC000E90FF11D877021E030E0A90102C0440F26
:103DD000551F8A95E2F7CA018095918189238183D5
:103DE00008959091DF0190FF16C01F928F938FEB83
:103DF00094E09F938F930E9405070F900F900F9070
:103E00000F9008953196E217F30729F090819813E7
:103E1000F9CF1082F7CF089581E090E0E0910D0195
:103E2000F0910E01E80FF91F108201968031910583
:103E3000A9F708959091DE01892B8093DE01089502
:103E400080959091DE0189238093DE010895109280
:103E5000DE0108959091DD01892B8093DD010895A5
:103E600080959091DD0189238093DD010895109262
:103E7000DD0108959091DC01892B8093DC01089588
:103E800080959091DC0189238093DC010895109244
:103E9000DC0108958093CB0108951092CB01089521
:103EA00080910D0190910E01FC0131969C01205FE3
:103EB0003F4F80E0919191118F5FE217F307D1F7A7
:103EC0000895E0910D01F0910E018091DE01808353
:103ED000E0910D01F0910E0190818091DD01892B1F
:103EE0008083E0910D01F0910E0190818091DC01C1
:103EF000892B80838091CB01882361F0E0910D01B3
:103F0000F0910E019081892B80830E94501F8111B6
:103F10001092CB0180910D0190910E010C94F01341
:103F20009093490180934801089520E0009739F06B
:103F3000AC0141505109842395232F5FF7CF822F85
:103F400008958295982F9C7C392F36953695282F89
:103F5000237344E0249FC0011124932F982B292F11
:103F60002A7A2695892F8575880F822B08951F93AD
:103F7000CF93DF931F92CDB7DEB799830E94A11F25
:103F8000182F9981892F0E94A11F212F30E0322FF5
:103F90002227A901482BCA010F90DF91CF911F91D1
:103FA00008958091F401843021F11092E00120E421
:103FB00088E190E00FB6F894A895809360000FBE5A
:103FC0002093600080E00E94DC0A83B7817F8460D8
:103FD00083BF83B7816083BF7894889583B78E7FD2
:103FE00083BF88E10FB6F894809360001092600060
:103FF0000FBE0895089508950E94FA1F0E94370B7E
:104000000E94FB1F0E940B0C91E0811101C090E007
:10401000892F08950E94FA180E94E4130C94DC0A78
:104020001F920F920FB60F9211248F939F93AF930D
:10403000BF938091E001811113C08091E1019091C3
:10404000E201A091E301B091E4014196A11DB11DEF
:104050008093E1019093E201A093E301B093E40126
:10406000BF91AF919F918F910F900FBE0F901F90B6
:10407000189582E084BD93E095BD9AEF97BD80933B
:104080006E0008952FB7F8948091E1019091E201BC
:10409000A091E301B091E4012FBF0895CF92DF9288
:1040A000EF92FF920F931F932FB7F8944091E10185
:1040B0005091E2016091E3017091E4012FBF6A0128
:1040C0007B01EE24FF248C0120E030E0C016D106F5
:1040D000E206F30610F4415051099A01281B390BEE
:1040E000C9011F910F91FF90EF90DF90CF9008953D
:1040F0001F920F920FB60F9211248F939F93AF933D
:10410000BF938091E1019091E201A091E301B09110
:10411000E4010196A11DB11D8093E1019093E2019C
:10412000A093E301B093E401BF91AF919F918F9170
:104130000F900FBE0F901F9018950E94E210F894F8
:104140002FEF87EA91E6215080409040E1F700C0D0
:10415000000087E090EBDC018093FE019093FF016B
:10416000A0930002B09301029CE088E10FB6F8949E
:10417000A895809360000FBE90936000FFCF0E94CF
:10418000F420811102C00E94DA200E94FF20809357
:10419000DF010E9407218093FD0187FB882780F9BA
:1041A00080930C010E940321682F70E080E090E072
:1041B0000C94BA1C6DEE7EEF80E090E00E943429F2
:1041C00060E082E090E00E94222960E083E090E0DD
:1041D0000E94222960E084E090E00E94222960E0B1
:1041E00085E090E00C94222980E090E00E941C2958
:1041F00021E08D3E9E4F09F020E0822F089582E05D
:1042000090E00C94142983E090E00C94142984E04D
:1042100090E00C941429682F84E090E00C942229FB
:104220008091E70180FF0BC06091120185E0689FDB
:10423000B001112475956795759567952BC081FF21
:1042400009C06091120185E0689FB0011124759545
:10425000679520C082FF07C06091120185E0689FCA
:10426000B001112417C09091E8019923D1F0609119
:104270001101961788F72091120185E0289F90017F
:104280001124929FA001939F500D112470E0CA0148
:104290000E94E6286038710540F46115710539F017
:1042A00002C065E070E0862F08958FE7089581E0F1
:1042B00008958091E70180FF08C06091100170E0CF
:1042C000759567957595679521C081FF06C06091CA
:1042D000100170E07595679519C082FF04C0609168
:1042E000100170E010C09091E8019923C1F0609135
:1042F0000F019617A0F780911001899FC00111242A
:1043000070E00E94E6286038710528F46115710597
:1043100021F0862F08958FE7089581E0089561E0E8
:1043200070E0F4CF803F21F40E941021819504C0F9
:10433000813F29F40E9410218093EB010895823F70
:1043400021F40E941021819504C0833F29F40E942A
:1043500010218093EA010895893F19F40E945921A0
:1043600005C08A3F31F40E94592181958093EC0168
:1043700008958B3F21F40E945921819504C08C3F00
:1043800029F40E9459218093ED010895843F21F47E
:104390008091E901816017C0853F21F48091E90196
:1043A000826011C0863F21F48091E90184600BC0D6
:1043B000873F21F48091E901886005C0883F31F48E
:1043C0008091E90180618093E90108958D3F21F496
:1043D0008091E70181600BC08E3F21F48091E7015D
:1043E000826005C08F3F29F48091E701846080934B
:1043F000E7010895803F39F48091EB0187FF6CC09D
:104400001092EB0169C0813F29F48091EB011816ED
:10441000BCF362C09091EA01823F29F497FF5CC02F
:104420001092EA0159C0833F19F41916CCF354C015
:10443000893F41F48091EC0118160CF04DC01092A8
:10444000EC014AC08A3F29F48091EC0187FF44C007
:10445000F6CF8B3F39F48091ED0187FF3DC010927C
:10446000ED013AC08C3F29F48091ED011816BCF3A0
:1044700033C0843F21F48091E9018E7F17C0853FCE
:1044800021F48091E9018D7F11C0863F21F4809154
:10449000E9018B7F0BC0873F21F48091E901877F81
:1044A00005C0883F31F48091E9018F7E8093E90156
:1044B00013C08D3F21F48091E7018E7F0BC08E3FAA
:1044C00021F48091E7018D7F05C08F3F29F4809111
:1044D000E7018B7F8093E7018091EA0181110EC093
:1044E0008091EB0181110AC08091EC01811106C01D
:1044F0008091ED01811102C01092E8010895809130
:10450000DF0183FF7EC082E295E00E946C0680910D
:10451000E9011F928F938DE195E09F938F930E9405
:1045200005078BE195E00E946C068091EA01282F37
:10453000332727FD30953F938F9388E195E09F9334
:104540008F930E94050786E195E00E946C0680919A
:10455000EB01282F332727FD30953F938F9383E17D
:1045600095E09F938F930E94050781E195E00E945B
:104570006C068091EC01282F332727FD30953F935F
:104580008F938EE095E09F938F930E9405078CE0B8
:1045900095E00E946C068091ED01282F332727FDBE
:1045A00030953F938F9389E095E09F938F930E947E
:1045B000050786E095E00E946C068091E8011F9255
:1045C0008F9383E095E09F938F930E94050781E08E
:1045D00095E00E946C068091E7011F928F938EEF09
:1045E00094E09F938F930E9405078BEF94E00E94C5
:1045F0006C068DB79EB74C960FB6F8949EBF0FBE53
:104600008DBF89EE91E00E9439140E944220909360
:10461000E6018093E50108951F93CF93DF93809186
:10462000E5019091E6010E944E20AC019091E801D5
:10463000992321F02091130130E006C0209114014C
:104640008AE0289F900111244217530708F486C07E
:104650008091EA01C091EB01D091EC011091ED0144
:10466000811107C0C11176C0D11174C0111172C07F
:1046700075C09F3F19F09F5F9093E801181624F4CE
:104680000E9410218093EA018091EA0187FF05C012
:104690000E94102181958093EA011C1624F40E9447
:1046A00010218093EB018091EB0187FF05C00E94F0
:1046B000102181958093EB016091EA01662339F125
:1046C000C091EB01CC2319F1772767FD7095872FF7
:1046D000972F0E94EB2723E333E343E35FE30E943A
:1046E0004F280E94B8276093EA016C2F772767FD57
:1046F0007095872F972F0E94EB2723E333E343E343
:104700005FE30E944F280E94B8276093EB011D16BB
:1047100024F40E9459218093EC018091EC0187FFE1
:1047200005C00E94592181958093EC01111624F453
:104730000E9459218093ED018091ED0187FF05C012
:104740000E94592181958093ED01DF91CF911F91B6
:104750000C947F229F3F09F08ECF96CFDF91CF91AF
:104760001F910895E9EEF1E085E0DF011D928A9541
:10477000E9F71092E8011092E701089585E497E0C7
:104780000E946C061F9281E08F931F9285E08F93A9
:1047900087EF96E09F938F930E9405070F900F90ED
:1047A0000F900F900F900F9008958330E9F128F447
:1047B000813061F0823009F10895853009F462C0DA
:1047C00008F449C0863009F474C00895809114013A
:1047D000262F30E0280F311D2F3F310524F4680FBC
:1047E0006093140103C08FEF809314018091140132
:1047F0001F928F9380E396E072C080911301262F61
:1048000030E0280F311D2F3F310524F4680F6093ED
:10481000130103C08FEF80931301809113011F9246
:104820008F938EE196E05BC080911201262F30E0DD
:10483000280F311D2F3F310524F4680F60931201BA
:1048400003C08FEF80931201809112011F928F930A
:104850008BE096E044C080911101262F30E0280FB4
:10486000311D2F3F310524F4680F6093110103C0FF
:104870008FEF80931101809111011F928F9386EF2A
:1048800095E02DC080911001262F30E0280F311DBA
:104890002F3F310524F4680F6093100103C08FEFA0
:1048A00080931001809110011F928F938DED95E000
:1048B00016C080910F01262F30E0280F311D2F3FA9
:1048C000310524F4680F60930F0103C08FEF8093CC
:1048D0000F0180910F011F928F9382EC95E09F93BF
:1048E0008F930E9405070F900F900F900F900895DF
:1048F000833081F128F4813059F08230D1F008956D
:10490000853009F449C0B8F1863009F456C00895DD
:1049100080911401681720F4861B8093140102C053
:1049200010921401809114011F928F9383EB95E0F4
:1049300054C080911301681720F4861B80931301E3
:1049400002C010921301809113011F928F9381EA8C
:1049500095E043C080911201681720F4861B809374
:10496000120102C010921201809112011F928F93C6
:104970008EE895E032C080911101681720F4861B03
:104980008093110102C010921101809111011F92B8
:104990008F9389E795E021C080911001681720F47A
:1049A000861B8093100102C01092100180911001AB
:1049B0001F928F9380E695E010C080910F016817D9
:1049C00020F4861B80930F0102C010920F0180918A
:1049D0000F011F928F9385E495E09F938F930E9420
:1049E00005070F900F900F900F900895CF93C82F49
:1049F0001F928F938AE498E09F938F930E940507FC
:104A000081E090E0A0E0B0E0BC01CD0104C0660F01
:104A1000771F881F991FCA95D2F70E94BA1C0F9062
:104A20000F900F900F90CF910C94FA18CF9387327C
:104A3000A8F58E3108F035C1803109F4A5C0F8F42D
:104A4000873009F465C0A8F4863009F030C1809140
:104A5000DF01817F8E7F8093DF018FEC99E00E94E0
:104A60006C0680E39CE00E946C0681E08093EF017D
:104A70004DC08B30F1F18E3009F472C018C186310F
:104A800009F4B6C020F4813109F4F9C010C18931AC
:104A900009F497C08B3109F44FC009C1883349F13B
:104AA00050F4893209F4FFC0853309F4FCC0873221
:104AB00009F4F9C0FCC0833409F4F5C028F48A3342
:104AC00008F4F5C08953F0C0883409F0F0C00E94A2
:104AD000FA1884E19CE00E946C062FEF83ED90E3CE
:104AE000215080409040E1F700C000000E949D20CE
:104AF0000DC086EF99E062C08BEF9BE00E946C06D0
:104B00008091DF01897F877F8093DF01C1E0D4C07E
:104B10008091DF01C82FC095C170C0FB80F98093E0
:104B2000DF01CC2349F388E09CE00E946C06809171
:104B3000DF01866088603DC09091DF0191FBCC274A
:104B4000C0F981E0C827892FC0FB81F98093DF017C
:104B5000CC2319F08EEE9BE027C080EE9BE02EC0A8
:104B60009091DF0192FBCC27C0F981E0C827892F03
:104B7000C0FB82F98093DF01CC2319F081ED9BE02B
:104B800013C081EC9BE01AC09091DF0193FBCC270E
:104B9000C0F981E0C827892FC0FB83F98093DF012A
:104BA000CC2351F085EB9BE00E946C068091DF01E5
:104BB00081608093DF0180C088EA9BE00E946C06E0
:104BC000A5CF80EC99E00E946C0685E999E00E94EF
:104BD0006C068BE599E00E946C068EE299E00E94DB
:104BE0006C0683EF98E00E946C0688EC98E0E6CFB4
:104BF0008AEB98E00E946C060E94E4131F928F9348
:104C000080EA98E09F938F930E94050780910B01A3
:104C10001F928F9389E898E09F938F930E940507D6
:104C200080917A011F928F9386E798E09F938F93EC
:104C30000E94050780910C011F928F9383E698E0F4
:104C40009F938F930E9405078091E1019091E2016B
:104C5000A091E301B091E401BF93AF939F938F9331
:104C60008FE498E09F938F930E9405078DB79EB7BE
:104C700046960FB6F8949EBF0FBE8DBF47CF0E94D9
:104C8000FA18C0910C0181E0C827C0930C01CC2315
:104C900029F08EE99BE00E946C060EC083E99BE040
:104CA0008DCF8D5101C080E00E94F6242FCF81E985
:104CB0009BE00E946C06C0E08C2FCF91089580E0AD
:104CC000089580E00895CF93C82F8091EF0181303F
:104CD00071F020F0823009F44BC042C1E0910D0127
:104CE000F0910E018081823209F03CC107C0E09151
:104CF0000D01F0910E018081823261F48C2F0E94AF
:104D00005F26811104C08C2F0E9416252FC081E0E0
:104D100090E02CC08C2F0E946126811126C0C431E6
:104D2000E1F070F4CB3081F0C031D1F40E94BE23A9
:104D300082E498E00E946C0682E08093EF0115C047
:104D4000C93259F0C83361F48FEC99E00E946C06C7
:104D500086E498E00E946C0608C01092EF0104C13E
:104D600080E498E00E946C06FFC081E08170FEC084
:104D7000C43228F5CE3108F0C1C0CB30A1F1D0F457
:104D8000C73009F0D3C08EE18093140182E3809391
:104D900013018AE08093120184E18093110188E07D
:104DA0008093100188E280930F0186EE96E00E94C6
:104DB0006C06BFC0C33149F1C431C1F0B7C0CB34B8
:104DC00009F4A9C028F4C93289F0C83361F0AEC033
:104DD000C13509F49EC0C23509F499C0CE3409F03A
:104DE000A5C06AE09EC00E94BE23A3C08091EE01D0
:104DF000882319F01092EE019CC083EF96E00E9488
:104E00006C0681E08093EF01B1C08DEC96E00E94CA
:104E10006C068BEB96E00E946C06809114011F9249
:104E20008F9388EB96E09F938F930E94050786EB04
:104E300096E00E946C0684EA96E00E946C068091DF
:104E400013011F928F9381EA96E09F938F930E94A4
:104E500005078FE996E00E946C0680E996E00E94C3
:104E60006C06809112011F928F938DE896E09F93BC
:104E70008F930E9405078BE896E00E946C068AE7F4
:104E800096E00E946C06809111011F928F9387E734
:104E900096E09F938F930E94050785E796E00E9416
:104EA0006C0680E696E00E946C06809110011F92CD
:104EB0008F938DE596E09F938F930E9405078BE576
:104EC00096E00E946C0684E496E00E946C06809155
:104ED0000F011F928F9381E496E09F938F930E941E
:104EE00005078FE396E00E946C068DB79EB7489643
:104EF0000FB6F8949EBF0FBE8DBF1BC0CE51EC2FD6
:104F0000F0E0E35CFE4F80818093EE0112C061E02F
:104F100003C061E006C06AE08091EE010E94D523E3
:104F200008C08091EE010E94782403C084EE96E0D0
:104F300013C08091EE01882369F01F928F938EED4C
:104F400096E09F938F930E9405070F900F900F900C
:104F50000F9004C08BED96E00E946C0681E006C0C5
:104F60001092EF0180E002C080E000CFCF91089561
:104F700004D06894B1118DC0089570D088F09F5707
:104F800090F0B92F9927B751A0F0D1F0660F771F95
:104F9000881F991F1AF0BA95C9F712C0B13081F075
:104FA00077D0B1E0089574C0672F782F8827B85F55
:104FB00039F0B93FCCF3869577956795B395D9F7D6
:104FC0003EF490958095709561957F4F8F4F9F4FE0
:104FD0000895E89409C097FB3EF4909580957095EC
:104FE00061957F4F8F4F9F4F9923A9F0F92F96E935
:104FF000BB279395F695879577956795B795F111AA
:10500000F8CFFAF4BB0F11F460FF1BC06F5F7F4F46
:105010008F4F9F4F16C0882311F096E911C0772358
:1050200021F09EE8872F762F05C0662371F096E861
:10503000862F70E060E02AF09A95660F771F881F30
:10504000DAF7880F9695879597F9089557FD905848
:10505000440F551F59F05F3F71F04795880F97FB3C
:10506000991F61F09F3F79F08795089512161306F6
:105070001406551FF2CF4695F1DF08C01616170625
:105080001806991FF1CF869571056105089408955A
:10509000E894BB2766277727CB0197F908950BD0B3
:1050A00078C069D028F06ED018F0952309F05AC066
:1050B0005FC01124EECFCADFA0F3959FD1F3950F07
:1050C00050E0551F629FF001729FBB27F00DB11D8C
:1050D000639FAA27F00DB11DAA1F649F6627B00D1C
:1050E000A11D661F829F2227B00DA11D621F739F05
:1050F000B00DA11D621F839FA00D611D221F749F13
:105100003327A00D611D231F849F600D211D822F59
:10511000762F6A2F11249F5750408AF0E1F08823A0
:105120004AF0EE0FFF1FBB1F661F771F881F9150AD
:105130005040A9F79E3F510570F014C0AACF5F3FC1
:10514000ECF3983EDCF3869577956795B795F795E0
:10515000E7959F5FC1F7FE2B880F911D9695879568
:1051600097F9089597F99F6780E870E060E00895E7
:105170009FEF80EC089500240A941616170618066F
:105180000906089500240A9412161306140605064B
:105190000895092E0394000C11F4882352F0BB0FDC
:1051A00040F4BF2B11F460FF04C06F5F7F4F8F4F3F
:1051B0009F4F0895991B79E004C0991F961708F036
:1051C000961B881F7A95C9F78095089597FB072E3F
:1051D00016F4009407D077FD09D00E94002907FC3F
:1051E00005D03EF4909581959F4F089570956195F7
:1051F0007F4F0895EE0FFF1F0590F491E02D099465
:10520000AA1BBB1B51E107C0AA1FBB1FA617B707EC
:1052100010F0A61BB70B881F991F5A95A9F7809508
:105220009095BC01CD010895F999FECF92BD81BD45
:10523000F89A992780B50895A8E1B0E042E050E0DF
:105240000C943C29262FF999FECF92BD81BDF89A86
:10525000019700B4021639F01FBA20BD0FB6F894BA
:10526000FA9AF99A0FBE08950196272F0E942329D2
:105270000C942229DC01CB01FC01F999FECF06C078
:10528000F2BDE1BDF89A319600B40D924150504004
:08529000B8F70895F894FFCF70
:10529800FF210C120DEF0CBB0C870C0101CC01286F
:1052A80008140A321E796653436C49636F7F697329
:1052B800091939293F4D3620394D040004CA03AA7B
:1052C800037103E402FD0216032F034F03010203D7
:0852D8000405060708090000A7
:00000001FF
